 management

 Timestamp is 6a163892 (Tue May 26 20:19:30 2026)

 Preferred load address is 10000000

 Start         Length     Name                   Class
 0001:00000000 000010e1H .text$mn                CODE
 0002:00000000 000000c8H .idata$5                DATA
 0002:000000c8 00000008H .00cfg                  DATA
 0002:000000d0 00000004H .CRT$XCA                DATA
 0002:000000d4 00000004H .CRT$XCZ                DATA
 0002:000000d8 00000004H .CRT$XIA                DATA
 0002:000000dc 00000004H .CRT$XIZ                DATA
 0002:000000e0 00000004H .CRT$XPA                DATA
 0002:000000e4 00000004H .CRT$XPZ                DATA
 0002:000000e8 00000004H .CRT$XTA                DATA
 0002:000000ec 00000004H .CRT$XTZ                DATA
 0002:000000f0 00000000H .gfids$y                DATA
 0002:000000f0 00000250H .rdata                  DATA
 0002:00000340 00000000H .rdata$CastGuardVftablesA DATA
 0002:00000340 00000000H .rdata$CastGuardVftablesC DATA
 0002:00000340 00000004H .rdata$sxdata           DATA
 0002:00000344 00000064H .rdata$voltmd           DATA
 0002:000003a8 000002f8H .rdata$zzzdbg           DATA
 0002:000006a0 00000004H .rtc$IAA                DATA
 0002:000006a4 00000004H .rtc$IZZ                DATA
 0002:000006a8 00000004H .rtc$TAA                DATA
 0002:000006ac 00000004H .rtc$TZZ                DATA
 0002:000006b0 00000090H .xdata$x                DATA
 0002:00000740 00000110H .edata                  DATA
 0002:00000850 000000a0H .idata$2                DATA
 0002:000008f0 00000014H .idata$3                DATA
 0002:00000904 000000c8H .idata$4                DATA
 0002:000009cc 00000456H .idata$6                DATA
 0003:00000000 00000018H .data                   DATA
 0003:00000018 0000037cH .bss                    DATA
 0004:00000000 00000060H .rsrc$01                DATA
 0004:00000060 00000378H .rsrc$02                DATA

  Address         Publics by Value              Rva+Base       Lib:Object

 0000:00000000       ___AbsoluteZero            00000000     <absolute>
 0000:00000000       ___arm64x_extra_rfe_table  00000000     <absolute>
 0000:00000000       ___arm64x_extra_rfe_table_size 00000000     <absolute>
 0000:00000000       ___arm64x_native_entrypoint 00000000     <absolute>
 0000:00000000       ___arm64x_redirection_metadata 00000000     <absolute>
 0000:00000000       ___arm64x_redirection_metadata_count 00000000     <absolute>
 0000:00000000       ___dynamic_value_reloc_table 00000000     <absolute>
 0000:00000000       ___enclave_config          00000000     <absolute>
 0000:00000000       ___guard_check_icall_a64n_fptr 00000000     <absolute>
 0000:00000000       ___guard_eh_cont_count     00000000     <absolute>
 0000:00000000       ___guard_eh_cont_table     00000000     <absolute>
 0000:00000000       ___guard_fids_count        00000000     <absolute>
 0000:00000000       ___guard_fids_table        00000000     <absolute>
 0000:00000000       ___guard_iat_count         00000000     <absolute>
 0000:00000000       ___guard_iat_table         00000000     <absolute>
 0000:00000000       ___guard_longjmp_count     00000000     <absolute>
 0000:00000000       ___guard_longjmp_table     00000000     <absolute>
 0000:00000000       ___hybrid_auxiliary_iat    00000000     <absolute>
 0000:00000000       ___hybrid_auxiliary_iat_copy 00000000     <absolute>
 0000:00000000       ___hybrid_code_map         00000000     <absolute>
 0000:00000000       ___hybrid_code_map_count   00000000     <absolute>
 0000:00000000       ___x64_code_ranges_to_entry_points 00000000     <absolute>
 0000:00000000       ___x64_code_ranges_to_entry_points_count 00000000     <absolute>
 0000:00000001       ___safe_se_handler_count   00000001     <absolute>
 0000:00000100       ___guard_flags             00000100     <absolute>
 0000:00000000       ___ImageBase               10000000     <linker-defined>
 0001:00000000       _Java_sun_management_FileSystemImpl_init0@8 10001000 f   FileSystemImpl.obj
 0001:00000003       _Java_sun_management_FileSystemImpl_isAccessUserOnly0@12 10001003 f   FileSystemImpl.obj
 0001:0000009d       _Java_sun_management_FileSystemImpl_isSecuritySupported0@12 1000109d f   FileSystemImpl.obj
 0001:00000349       _JNI_OnLoad@8              10001349 f   management.obj
 0001:000003a7       ___local_stdio_printf_options 100013a7 f i management.obj
 0001:000003ad       _JVM_GetManagement@4       100013ad f   jvm:jvm.dll
 0001:000003b3       _JNU_ThrowOutOfMemoryError@8 100013b3 f   java:java.dll
 0001:000003b9       _JNU_ThrowInternalError@8  100013b9 f   java:java.dll
 0001:000003bf       _JNU_ThrowIOException@8    100013bf f   java:java.dll
 0001:000003c5       _JNU_ThrowIOExceptionWithLastError@8 100013c5 f   java:java.dll
 0001:000003cb       _JNU_GetStringPlatformChars@12 100013cb f   java:java.dll
 0001:000003d1       _JNU_ReleaseStringPlatformChars@12 100013d1 f   java:java.dll
 0001:000003d7       @__security_check_cookie@4 100013d7 f   MSVCRT:secchk.obj
 0001:00000725       __DllMainCRTStartup@12     10001725 f   MSVCRT:dll_dllmain.obj
 0001:00000748       ___raise_securityfailure   10001748 f   MSVCRT:gs_report.obj
 0001:00000770       ___report_gsfailure        10001770 f   MSVCRT:gs_report.obj
 0001:000008b7       ___security_init_cookie    100018b7 f   MSVCRT:gs_support.obj
 0001:00000902       _DllMain@12                10001902 f   MSVCRT:dll_dllmain_stub.obj
 0001:00000924       ?__scrt_initialize_type_info@@YAXXZ 10001924 f   MSVCRT:tncleanup.obj
 0001:00000930       ?__scrt_uninitialize_type_info@@YAXXZ 10001930 f   MSVCRT:tncleanup.obj
 0001:0000093c       ___local_stdio_scanf_options 1000193c f i MSVCRT:default_local_stdio_options.obj
 0001:00000942       ___scrt_initialize_default_local_stdio_options 10001942 f   MSVCRT:default_local_stdio_options.obj
 0001:000009a3       ___scrt_acquire_startup_lock 100019a3 f   MSVCRT:utility.obj
 0001:000009d5       ___scrt_dllmain_after_initialize_c 100019d5 f   MSVCRT:utility.obj
 0001:00000a00       ___scrt_dllmain_before_initialize_c 10001a00 f   MSVCRT:utility.obj
 0001:00000a0e       ___scrt_dllmain_crt_thread_attach 10001a0e f   MSVCRT:utility.obj
 0001:00000a2d       ___scrt_dllmain_crt_thread_detach 10001a2d f   MSVCRT:utility.obj
 0001:00000a3a       ___scrt_dllmain_exception_filter 10001a3a f   MSVCRT:utility.obj
 0001:00000a6e       ___scrt_dllmain_uninitialize_c 10001a6e f   MSVCRT:utility.obj
 0001:00000a91       ___scrt_dllmain_uninitialize_critical 10001a91 f   MSVCRT:utility.obj
 0001:00000a9e       ___scrt_initialize_crt     10001a9e f   MSVCRT:utility.obj
 0001:00000ad7       ___scrt_initialize_onexit_tables 10001ad7 f   MSVCRT:utility.obj
 0001:00000b5e       ___scrt_is_nonwritable_in_current_image 10001b5e f   MSVCRT:utility.obj
 0001:00000bf2       ___scrt_release_startup_lock 10001bf2 f   MSVCRT:utility.obj
 0001:00000c0f       ___scrt_uninitialize_crt   10001c0f f   MSVCRT:utility.obj
 0001:00000c37       ___scrt_get_dyn_tls_init_callback 10001c37 f   MSVCRT:dyn_tls_init.obj
 0001:00000c3d       ___scrt_fastfail           10001c3d f   MSVCRT:utility_desktop.obj
 0001:00000d58       __crt_debugger_hook        10001d58 f   MSVCRT:utility_desktop.obj
 0001:00000d60       __RTC_Initialize           10001d60 f   MSVCRT:initsect.obj
 0001:00000d8c       __RTC_Terminate            10001d8c f   MSVCRT:initsect.obj
 0001:00000dc0       __SEH_prolog4              10001dc0 f   MSVCRT:sehprolg4.obj
 0001:00000e05       __except_handler4          10001e05 f   MSVCRT:chandler4gs.obj
 0001:00000e34       @_guard_check_icall_nop@4  10001e34 f i MSVCRT:guard_support.obj
 0001:00000e37       ___isa_available_init      10001e37 f   MSVCRT:cpu_disp.obj
 0001:0000100b       __get_startup_argv_mode    1000200b f   MSVCRT:argv_mode.obj
 0001:0000100f       ___scrt_is_ucrt_dll_in_use 1000200f f   MSVCRT:ucrt_detection.obj
 0001:0000101b       _strchr                    1000201b f   vcruntime:VCRUNTIME140.dll
 0001:00001021       ___std_type_info_destroy_list 10002021 f   vcruntime:VCRUNTIME140.dll
 0001:00001027       _memset                    10002027 f   vcruntime:VCRUNTIME140.dll
 0001:0000102d       __except_handler4_common   1000202d f   vcruntime:VCRUNTIME140.dll
 0001:00001033       __initterm                 10002033 f   ucrt:api-ms-win-crt-runtime-l1-1-0.dll
 0001:00001039       __initterm_e               10002039 f   ucrt:api-ms-win-crt-runtime-l1-1-0.dll
 0001:0000103f       __seh_filter_dll           1000203f f   ucrt:api-ms-win-crt-runtime-l1-1-0.dll
 0001:00001045       __configure_narrow_argv    10002045 f   ucrt:api-ms-win-crt-runtime-l1-1-0.dll
 0001:0000104b       __initialize_narrow_environment 1000204b f   ucrt:api-ms-win-crt-runtime-l1-1-0.dll
 0001:00001051       __initialize_onexit_table  10002051 f   ucrt:api-ms-win-crt-runtime-l1-1-0.dll
 0001:00001057       __execute_onexit_table     10002057 f   ucrt:api-ms-win-crt-runtime-l1-1-0.dll
 0001:0000105d       __cexit                    1000205d f   ucrt:api-ms-win-crt-runtime-l1-1-0.dll
 0001:00001063       ___acrt_initialize         10002063 f   MSVCRT:ucrt_stubs.obj
 0001:00001063       ___acrt_thread_attach      10002063 f   MSVCRT:ucrt_stubs.obj
 0001:00001063       ___acrt_thread_detach      10002063 f   MSVCRT:ucrt_stubs.obj
 0001:00001063       ___acrt_uninitialize       10002063 f   MSVCRT:ucrt_stubs.obj
 0001:00001063       ___acrt_uninitialize_critical 10002063 f   MSVCRT:ucrt_stubs.obj
 0001:00001063       ___scrt_stub_for_acrt_initialize 10002063 f   MSVCRT:ucrt_stubs.obj
 0001:00001063       ___scrt_stub_for_acrt_thread_attach 10002063 f   MSVCRT:ucrt_stubs.obj
 0001:00001063       ___scrt_stub_for_acrt_thread_detach 10002063 f   MSVCRT:ucrt_stubs.obj
 0001:00001063       ___scrt_stub_for_acrt_uninitialize 10002063 f   MSVCRT:ucrt_stubs.obj
 0001:00001063       ___scrt_stub_for_acrt_uninitialize_critical 10002063 f   MSVCRT:ucrt_stubs.obj
 0001:00001063       ___vcrt_initialize         10002063 f   MSVCRT:ucrt_stubs.obj
 0001:00001063       ___vcrt_thread_attach      10002063 f   MSVCRT:ucrt_stubs.obj
 0001:00001063       ___vcrt_thread_detach      10002063 f   MSVCRT:ucrt_stubs.obj
 0001:00001063       ___vcrt_uninitialize       10002063 f   MSVCRT:ucrt_stubs.obj
 0001:00001063       ___vcrt_uninitialize_critical 10002063 f   MSVCRT:ucrt_stubs.obj
 0001:00001066       ___scrt_stub_for_is_c_termination_complete 10002066 f   MSVCRT:ucrt_stubs.obj
 0001:00001066       __is_c_termination_complete 10002066 f   MSVCRT:ucrt_stubs.obj
 0001:00001069       __filter_x86_sse2_floating_point_exception 10002069 f   MSVCRT:x86_exception_filter.obj
 0001:00001069       __filter_x86_sse2_floating_point_exception_default 10002069 f   MSVCRT:x86_exception_filter.obj
 0002:00000000       __imp__GetSecurityDescriptorOwner@12 10003000     advapi32:ADVAPI32.dll
 0002:00000004       __imp__GetSecurityDescriptorDacl@16 10003004     advapi32:ADVAPI32.dll
 0002:00000008       __imp__GetAclInformation@16 10003008     advapi32:ADVAPI32.dll
 0002:0000000c       __imp__GetAce@12           1000300c     advapi32:ADVAPI32.dll
 0002:00000010       __imp__EqualSid@8          10003010     advapi32:ADVAPI32.dll
 0002:00000014       __imp__GetFileSecurityA@20 10003014     advapi32:ADVAPI32.dll
 0002:00000018       \177ADVAPI32_NULL_THUNK_DATA 10003018     advapi32:ADVAPI32.dll
 0002:0000001c       __imp__QueryPerformanceCounter@4 1000301c     kernel32:KERNEL32.dll
 0002:00000020       __imp__GetSystemTimeAsFileTime@4 10003020     kernel32:KERNEL32.dll
 0002:00000024       __imp__DisableThreadLibraryCalls@4 10003024     kernel32:KERNEL32.dll
 0002:00000028       __imp__InitializeSListHead@4 10003028     kernel32:KERNEL32.dll
 0002:0000002c       __imp__IsDebuggerPresent@0 1000302c     kernel32:KERNEL32.dll
 0002:00000030       __imp__GetCurrentProcessId@0 10003030     kernel32:KERNEL32.dll
 0002:00000034       __imp__GetCurrentThreadId@0 10003034     kernel32:KERNEL32.dll
 0002:00000038       __imp__GetVolumeInformationA@32 10003038     kernel32:KERNEL32.dll
 0002:0000003c       __imp__GetLastError@0      1000303c     kernel32:KERNEL32.dll
 0002:00000040       __imp__UnhandledExceptionFilter@4 10003040     kernel32:KERNEL32.dll
 0002:00000044       __imp__SetUnhandledExceptionFilter@4 10003044     kernel32:KERNEL32.dll
 0002:00000048       __imp__GetCurrentProcess@0 10003048     kernel32:KERNEL32.dll
 0002:0000004c       __imp__TerminateProcess@8  1000304c     kernel32:KERNEL32.dll
 0002:00000050       __imp__IsProcessorFeaturePresent@4 10003050     kernel32:KERNEL32.dll
 0002:00000054       \177KERNEL32_NULL_THUNK_DATA 10003054     kernel32:KERNEL32.dll
 0002:00000058       __imp___except_handler4_common 10003058     vcruntime:VCRUNTIME140.dll
 0002:0000005c       __imp____std_type_info_destroy_list 1000305c     vcruntime:VCRUNTIME140.dll
 0002:00000060       __imp__strchr              10003060     vcruntime:VCRUNTIME140.dll
 0002:00000064       __imp__memset              10003064     vcruntime:VCRUNTIME140.dll
 0002:00000068       \177VCRUNTIME140_NULL_THUNK_DATA 10003068     vcruntime:VCRUNTIME140.dll
 0002:0000006c       __imp__malloc              1000306c     ucrt:api-ms-win-crt-heap-l1-1-0.dll
 0002:00000070       __imp__free                10003070     ucrt:api-ms-win-crt-heap-l1-1-0.dll
 0002:00000074       \177api-ms-win-crt-heap-l1-1-0_NULL_THUNK_DATA 10003074     ucrt:api-ms-win-crt-heap-l1-1-0.dll
 0002:00000078       __imp___initialize_onexit_table 10003078     ucrt:api-ms-win-crt-runtime-l1-1-0.dll
 0002:0000007c       __imp___cexit              1000307c     ucrt:api-ms-win-crt-runtime-l1-1-0.dll
 0002:00000080       __imp___configure_narrow_argv 10003080     ucrt:api-ms-win-crt-runtime-l1-1-0.dll
 0002:00000084       __imp___initialize_narrow_environment 10003084     ucrt:api-ms-win-crt-runtime-l1-1-0.dll
 0002:00000088       __imp___seh_filter_dll     10003088     ucrt:api-ms-win-crt-runtime-l1-1-0.dll
 0002:0000008c       __imp___initterm           1000308c     ucrt:api-ms-win-crt-runtime-l1-1-0.dll
 0002:00000090       __imp___initterm_e         10003090     ucrt:api-ms-win-crt-runtime-l1-1-0.dll
 0002:00000094       __imp___execute_onexit_table 10003094     ucrt:api-ms-win-crt-runtime-l1-1-0.dll
 0002:00000098       \177api-ms-win-crt-runtime-l1-1-0_NULL_THUNK_DATA 10003098     ucrt:api-ms-win-crt-runtime-l1-1-0.dll
 0002:0000009c       __imp___strdup             1000309c     ucrt:api-ms-win-crt-string-l1-1-0.dll
 0002:0000009c       __imp__strdup              1000309c     ucrt:api-ms-win-crt-string-l1-1-0.dll
 0002:000000a0       \177api-ms-win-crt-string-l1-1-0_NULL_THUNK_DATA 100030a0     ucrt:api-ms-win-crt-string-l1-1-0.dll
 0002:000000a4       __imp__JNU_ReleaseStringPlatformChars@12 100030a4     java:java.dll
 0002:000000a8       __imp__JNU_GetStringPlatformChars@12 100030a8     java:java.dll
 0002:000000ac       __imp__JNU_ThrowIOExceptionWithLastError@8 100030ac     java:java.dll
 0002:000000b0       __imp__JNU_ThrowOutOfMemoryError@8 100030b0     java:java.dll
 0002:000000b4       __imp__JNU_ThrowInternalError@8 100030b4     java:java.dll
 0002:000000b8       __imp__JNU_ThrowIOException@8 100030b8     java:java.dll
 0002:000000bc       \177java_NULL_THUNK_DATA   100030bc     java:java.dll
 0002:000000c0       __imp__JVM_GetManagement@4 100030c0     jvm:jvm.dll
 0002:000000c4       \177jvm_NULL_THUNK_DATA    100030c4     jvm:jvm.dll
 0002:000000c8       ___guard_check_icall_fptr  100030c8     MSVCRT:guard_support.obj
 0002:000000cc       ___castguard_check_failure_os_handled_fptr 100030cc     MSVCRT:guard_support.obj
 0002:000000d0       ___xc_a                    100030d0     MSVCRT:initializers.obj
 0002:000000d4       ___xc_z                    100030d4     MSVCRT:initializers.obj
 0002:000000d8       ___xi_a                    100030d8     MSVCRT:initializers.obj
 0002:000000dc       ___xi_z                    100030dc     MSVCRT:initializers.obj
 0002:000000e0       ___xp_a                    100030e0     MSVCRT:initializers.obj
 0002:000000e4       ___xp_z                    100030e4     MSVCRT:initializers.obj
 0002:000000e8       ___xt_a                    100030e8     MSVCRT:initializers.obj
 0002:000000ec       ___xt_z                    100030ec     MSVCRT:initializers.obj
 0002:000000f0       ??_C@_0O@PNKFDMOJ@Malformed?5UNC@ 100030f0     FileSystemImpl.obj
 0002:00000100       ??_C@_0CA@CGFDCJE@Absolute?5filename?5not?5specified@ 10003100     FileSystemImpl.obj
 0002:00000120       ??_C@_0BM@JPGKFFDK@GetVolumeInformation?5failed@ 10003120     FileSystemImpl.obj
 0002:0000013c       ??_C@_0BH@EKMPGKNN@GetFileSecurity?5failed@ 1000313c     FileSystemImpl.obj
 0002:00000154       ??_C@_0CC@PLIGLKOL@GetSecurityDescriptorOwner?5fail@ 10003154     FileSystemImpl.obj
 0002:00000178       ??_C@_0CB@EKBMIJAO@GetSecurityDescriptorDacl?5faile@ 10003178     FileSystemImpl.obj
 0002:0000019c       ??_C@_0CM@JFCPAEMB@Security?5descriptor?5does?5not?5co@ 1000319c     FileSystemImpl.obj
 0002:000001c8       ??_C@_0BJ@OEDGCHLN@GetAclInformation?5failed@ 100031c8     FileSystemImpl.obj
 0002:000001e4       ??_C@_0O@HNKFIIOB@GetAce?5failed@ 100031e4     FileSystemImpl.obj
 0002:000001f4       ??_C@_0BP@KJIDAONK@Unsupported?5Management?5version@ 100031f4     management.obj
 0002:00000214       __pDefaultRawDllMain       10003214     MSVCRT:dll_dllmain.obj
 0002:00000214       __pRawDllMain              10003214     MSVCRT:dll_dllmain.obj
 0002:00000220       __load_config_used         10003220     MSVCRT:loadcfg.obj
 0002:00000340       ___safe_se_handler_table   10003340     <linker-defined>
 0002:00000344       ___volatile_metadata       10003344     <linker-defined>
 0002:000006a0       ___rtc_iaa                 100036a0     MSVCRT:initsect.obj
 0002:000006a4       ___rtc_izz                 100036a4     MSVCRT:initsect.obj
 0002:000006a8       ___rtc_taa                 100036a8     MSVCRT:initsect.obj
 0002:000006ac       ___rtc_tzz                 100036ac     MSVCRT:initsect.obj
 0002:00000850       __IMPORT_DESCRIPTOR_jvm    10003850     jvm:jvm.dll
 0002:00000864       __IMPORT_DESCRIPTOR_java   10003864     java:java.dll
 0002:00000878       __IMPORT_DESCRIPTOR_ADVAPI32 10003878     advapi32:ADVAPI32.dll
 0002:0000088c       __IMPORT_DESCRIPTOR_KERNEL32 1000388c     kernel32:KERNEL32.dll
 0002:000008a0       __IMPORT_DESCRIPTOR_VCRUNTIME140 100038a0     vcruntime:VCRUNTIME140.dll
 0002:000008b4       __IMPORT_DESCRIPTOR_api-ms-win-crt-heap-l1-1-0 100038b4     ucrt:api-ms-win-crt-heap-l1-1-0.dll
 0002:000008c8       __IMPORT_DESCRIPTOR_api-ms-win-crt-runtime-l1-1-0 100038c8     ucrt:api-ms-win-crt-runtime-l1-1-0.dll
 0002:000008dc       __IMPORT_DESCRIPTOR_api-ms-win-crt-string-l1-1-0 100038dc     ucrt:api-ms-win-crt-string-l1-1-0.dll
 0002:000008f0       __NULL_IMPORT_DESCRIPTOR   100038f0     jvm:jvm.dll
 0003:00000000       ___security_cookie_complement 10004000     MSVCRT:gs_cookie.obj
 0003:00000004       ___security_cookie         10004004     MSVCRT:gs_cookie.obj
 0003:00000008       ___scrt_native_dllmain_reason 10004008     MSVCRT:utility.obj
 0003:00000010       ___isa_enabled             10004010     MSVCRT:cpu_disp.obj
 0003:00000014       ___scrt_ucrt_dll_is_in_use 10004014     MSVCRT:ucrt_stubs.obj
 0003:00000018       _jmm_interface             10004018     management.obj
 0003:0000001c       _jmm_version               1000401c     management.obj
 0003:00000020       _jvm                       10004020     management.obj
 0003:00000348       ?__type_info_root_node@@3U__type_info_node@@A 10004348     MSVCRT:tncleanup.obj
 0003:00000350       ?_OptionsStorage@?1??__local_stdio_scanf_options@@9@4_KA 10004350     MSVCRT:default_local_stdio_options.obj
 0003:00000358       ___scrt_current_native_startup_state 10004358     MSVCRT:utility.obj
 0003:0000035c       ___scrt_native_startup_lock 1000435c     MSVCRT:utility.obj
 0003:0000037c       ___scrt_debugger_hook_flag 1000437c     MSVCRT:utility_desktop.obj
 0003:00000380       ___isa_available           10004380     MSVCRT:cpu_disp.obj
 0003:00000384       ___favor                   10004384     MSVCRT:cpu_disp.obj
 0003:00000388       ?_OptionsStorage@?1??__local_stdio_printf_options@@9@9 10004388     <common>
 0003:00000390       ___dyn_tls_init_callback   10004390     <common>

 entry point at        0001:00000725

 Static symbols

 0000:ffff9000       .debug$S                   10000000     management.exp
 0000:ffff9000       .debug$S                   10000000     vcruntime:VCRUNTIME140.dll
 0000:ffff9000       .debug$S                   10000000     vcruntime:VCRUNTIME140.dll
 0000:ffff9000       .debug$S                   10000000     vcruntime:VCRUNTIME140.dll
 0000:ffff9000       .debug$S                   10000000     vcruntime:VCRUNTIME140.dll
 0000:ffff9000       .debug$S                   10000000     vcruntime:VCRUNTIME140.dll
 0000:ffff9000       .debug$S                   10000000     vcruntime:VCRUNTIME140.dll
 0000:ffff9000       .debug$S                   10000000     ucrt:api-ms-win-crt-heap-l1-1-0.dll
 0000:ffff9000       .debug$S                   10000000     ucrt:api-ms-win-crt-heap-l1-1-0.dll
 0000:ffff9000       .debug$S                   10000000     ucrt:api-ms-win-crt-runtime-l1-1-0.dll
 0000:ffff9000       .debug$S                   10000000     ucrt:api-ms-win-crt-runtime-l1-1-0.dll
 0000:ffff9000       .debug$S                   10000000     ucrt:api-ms-win-crt-runtime-l1-1-0.dll
 0000:ffff9000       .debug$S                   10000000     ucrt:api-ms-win-crt-runtime-l1-1-0.dll
 0000:ffff9000       .debug$S                   10000000     ucrt:api-ms-win-crt-runtime-l1-1-0.dll
 0000:ffff9000       .debug$S                   10000000     ucrt:api-ms-win-crt-runtime-l1-1-0.dll
 0000:ffff9000       .debug$S                   10000000     ucrt:api-ms-win-crt-runtime-l1-1-0.dll
 0000:ffff9000       .debug$S                   10000000     ucrt:api-ms-win-crt-runtime-l1-1-0.dll
 0000:ffff9000       .debug$S                   10000000     ucrt:api-ms-win-crt-runtime-l1-1-0.dll
 0000:ffff9000       .debug$S                   10000000     ucrt:api-ms-win-crt-runtime-l1-1-0.dll
 0000:ffff9000       .debug$S                   10000000     ucrt:api-ms-win-crt-runtime-l1-1-0.dll
 0000:ffff9000       .debug$S                   10000000     ucrt:api-ms-win-crt-runtime-l1-1-0.dll
 0000:ffff9000       .debug$S                   10000000     ucrt:api-ms-win-crt-runtime-l1-1-0.dll
 0000:ffff9000       .debug$S                   10000000     ucrt:api-ms-win-crt-stdio-l1-1-0.dll
 0002:ffffd000       .idata$6                   10000000     ucrt:api-ms-win-crt-stdio-l1-1-0.dll
 0000:ffff9000       .debug$S                   10000000     ucrt:api-ms-win-crt-string-l1-1-0.dll
 0000:ffff9000       .debug$S                   10000000     advapi32:ADVAPI32.dll
 0000:ffff9000       .debug$S                   10000000     advapi32:ADVAPI32.dll
 0000:ffff9000       .debug$S                   10000000     advapi32:ADVAPI32.dll
 0000:ffff9000       .debug$S                   10000000     advapi32:ADVAPI32.dll
 0000:ffff9000       .debug$S                   10000000     advapi32:ADVAPI32.dll
 0000:ffff9000       .debug$S                   10000000     advapi32:ADVAPI32.dll
 0000:ffff9000       .debug$S                   10000000     kernel32:KERNEL32.dll
 0000:ffff9000       .debug$S                   10000000     kernel32:KERNEL32.dll
 0000:ffff9000       .debug$S                   10000000     kernel32:KERNEL32.dll
 0000:ffff9000       .debug$S                   10000000     kernel32:KERNEL32.dll
 0000:ffff9000       .debug$S                   10000000     kernel32:KERNEL32.dll
 0000:ffff9000       .debug$S                   10000000     kernel32:KERNEL32.dll
 0000:ffff9000       .debug$S                   10000000     kernel32:KERNEL32.dll
 0000:ffff9000       .debug$S                   10000000     kernel32:KERNEL32.dll
 0000:ffff9000       .debug$S                   10000000     kernel32:KERNEL32.dll
 0000:ffff9000       .debug$S                   10000000     kernel32:KERNEL32.dll
 0000:ffff9000       .debug$S                   10000000     kernel32:KERNEL32.dll
 0000:ffff9000       .debug$S                   10000000     kernel32:KERNEL32.dll
 0000:ffff9000       .debug$S                   10000000     kernel32:KERNEL32.dll
 0000:ffff9000       .debug$S                   10000000     kernel32:KERNEL32.dll
 0000:ffff9000       .debug$S                   10000000     kernel32:KERNEL32.dll
 0000:ffff9000       .debug$S                   10000000     kernel32:KERNEL32.dll
 0000:ffff9000       .debug$S                   10000000     jvm:jvm.dll
 0000:ffff9000       .debug$S                   10000000     java:java.dll
 0000:ffff9000       .debug$S                   10000000     java:java.dll
 0000:ffff9000       .debug$S                   10000000     java:java.dll
 0000:ffff9000       .debug$S                   10000000     java:java.dll
 0000:ffff9000       .debug$S                   10000000     java:java.dll
 0000:ffff9000       .debug$S                   10000000     java:java.dll
 0001:000000e3       _getFileDACL               100010e3 f   FileSystemImpl.obj
 0001:0000012d       _getFileSecurityDescriptor 1000112d f   FileSystemImpl.obj
 0001:000001b4       _isAccessUserOnly          100011b4 f   FileSystemImpl.obj
 0001:00000266       _isSecuritySupported       10001266 f   FileSystemImpl.obj
 0001:000003e5       ?dllmain_crt_dispatch@@YGHQAUHINSTANCE__@@KQAX@Z 100013e5 f   MSVCRT:dll_dllmain.obj
 0001:00000438       ?dllmain_crt_process_attach@@YAHQAUHINSTANCE__@@QAX@Z 10001438 f   MSVCRT:dll_dllmain.obj
 0001:0000053f       ?dllmain_crt_process_detach@@YAH_N@Z 1000153f f   MSVCRT:dll_dllmain.obj
 0001:000005ef       ?dllmain_dispatch@@YAHQAUHINSTANCE__@@KQAX@Z 100015ef f   MSVCRT:dll_dllmain.obj
 0001:000006fa       ?dllmain_raw@@YGHQAUHINSTANCE__@@KQAX@Z 100016fa f   MSVCRT:dll_dllmain.obj
 0001:0000086a       ___get_entropy             1000186a f   MSVCRT:gs_support.obj
 0001:0000095f       ?find_pe_section@@YAPAU_IMAGE_SECTION_HEADER@@QAEI@Z 1000195f f   MSVCRT:utility.obj
 0001:00000dc0       $$000000                   10001dc0     MSVCRT:sehprolg4.obj
 0002:00000218       _GS_ExceptionPointers      10003218     MSVCRT:gs_report.obj
 0002:000006b0       __sehtable$?dllmain_crt_process_attach@@YAHQAUHINSTANCE__@@QAX@Z 100036b0     MSVCRT:dll_dllmain.obj
 0002:000006d0       __sehtable$?dllmain_crt_process_detach@@YAH_N@Z 100036d0     MSVCRT:dll_dllmain.obj
 0002:000006f8       __sehtable$?dllmain_dispatch@@YAHQAUHINSTANCE__@@KQAX@Z 100036f8     MSVCRT:dll_dllmain.obj
 0002:00000718       __sehtable$___scrt_is_nonwritable_in_current_image 10003718     MSVCRT:utility.obj
 0002:00000740       .edata                     10003740     management.exp
 0002:00000768       rgpv                       10003768     management.exp
 0002:00000778       rgszName                   10003778     management.exp
 0002:00000788       rgwOrd                     10003788     management.exp
 0002:00000790       szName                     10003790     management.exp
 0002:0000079f       $N00001                    1000379f     management.exp
 0002:000007ad       $N00002                    100037ad     management.exp
 0002:000007d9       $N00003                    100037d9     management.exp
 0002:00000812       $N00004                    10003812     management.exp
 0002:000009e4       .idata$6                   100039e4     jvm:jvm.dll
 0002:00000ab2       .idata$6                   10003ab2     java:java.dll
 0002:00000b34       .idata$6                   10003b34     advapi32:ADVAPI32.dll
 0002:00000c8e       .idata$6                   10003c8e     kernel32:KERNEL32.dll
 0002:00000cea       .idata$6                   10003cea     vcruntime:VCRUNTIME140.dll
 0002:00000dbe       .idata$6                   10003dbe     ucrt:api-ms-win-crt-heap-l1-1-0.dll
 0002:00000dde       .idata$6                   10003dde     ucrt:api-ms-win-crt-runtime-l1-1-0.dll
 0002:00000e00       .idata$6                   10003e00     ucrt:api-ms-win-crt-string-l1-1-0.dll
 0003:00000024       ?__proc_attached@@3HA      10004024     MSVCRT:dll_dllmain.obj
 0003:00000028       _GS_ExceptionRecord        10004028     MSVCRT:gs_report.obj
 0003:00000078       _GS_ContextRecord          10004078     MSVCRT:gs_report.obj
 0003:00000360       ?is_initialized_as_dll@@3_NA 10004360     MSVCRT:utility.obj
 0003:00000361       ?module_local_atexit_table_initialized@@3_NA 10004361     MSVCRT:utility.obj
 0003:00000364       ?module_local_atexit_table@@3U_onexit_table_t@@A 10004364     MSVCRT:utility.obj
 0003:00000370       ?module_local_at_quick_exit_table@@3U_onexit_table_t@@A 10004370     MSVCRT:utility.obj
 0004:00000060       $R000000                   10005060     management.dll.res
